:020000040000FA
:040000005EEF00F0BF
:100018003180D8CF01F0E8CF02F0E0CF03F0F2A0B2
:1000280020D081CF04F004A82FA804D080500F0B53
:100038002B6E14D004AA2FAA04D080500F0B2A6E5E
:100048000DD004AC2FAC04D080500F0B296E06D015
:1000580004AE2FAE03D080500F0B286E04C02FF0D3
:10006800F290F0A205D0815080500F0B2C6EF092C8
:10007800F0A00DD08150040E3018D8B404D0030E6F
:100088003018D8A403D080500F0B2D6EF090F2A238
:1000980009D08150050E3018D8A403D080500F0B1A
:1000A8002D6EF29203C0E0FF02C0E8FF01C0D8FF46
:0800B800319010000EEF0AF078
:100600000001000A006400E8031027566172696166
:100610006E7428444950293A25642028256429000D
:100620004241444933352056657273696F6E202507
:1006300073002020207777772E6C6973792E64659C
:100640007600202020202025632563256325630074
:1006500020202020524541445900286E756C6C2999
:1006600000302E350000D388D38AD38CD396FC0E6D
:10067000D3169B9C000E0F01386F000E896E3F0E43
:10068000926E000E396F9368000E3A6FE00E946E12
:10069000000E3B6FF40E956E000E3C6F0F0E966EC3
:1006A000F19CF288F19AF086F198F088F2866288DF
:1006B000628A628C628EF28EF28C898E8C828C863B
:1006C00074EC08F0000E0101E46F000EE36F930E6E
:1006D000E325D96E010EE421DA6E200EDF6E8C0E5A
:1006E000E325E16E010EE421E26EDFCFE7FF850E28
:1006F000E325D96E010EE421DA6EE7CFDFFF7E0E2F
:10070000E325E16E010EE421E26EDFCFE7FFE34B6C
:10071000E42BE4BFDCD7E45104E1070EE35DD8A08D
:10072000D6D7000EE46F000EE36F690EE325D96E95
:10073000010EE421DA6E200EDF6E770EE325E16E06
:10074000010EE421E26EDFCFE7FF700EE325D96EE4
:10075000010EE421DA6EE7CFDFFFE34BE42BE4BFC9
:10076000E4D7E45104E1060EE35DD8A0DED7000E25
:10077000056E010E066E1F0E076E060E086E61EC0A
:1007800009F0150E056E010E066E1F0E076E060EA1
:10079000086E61EC09F02A0E056E010E066E1F0E42
:1007A000076E060E086E61EC09F03F0E056E010E35
:1007B000066E1F0E076E060E086E61EC09F0000E45
:1007C0000101E16FE18180BAE1910101E18384B02F
:1007D000E1930101E18584B2E1950BD0020E07D0CF
:1007E000030E05D0040E03D0050E01D0010E306EAD
:1007F0001ED00101E151010AD8B4F0D7030AD8B4E0
:10080000EFD7010AD8B4EAD7070AD8B4EBD7010A60
:10081000D8B4E4D7030AD8B4E7D7010AD8B4E4D7E8
:100820000F0AD8B4E1D7010AD8B4D8D7DFD784A447
:1008300002D0000E01D0010EE56F010E3EEC09F072
:10084000B00E116E010E126E200E136E060E146E97
:10085000610E156E060E166E25EC07F0000E096E81
:10086000000EA4EC09F0B00E096E010E0A6EC2EC87
:1008700009F0010E096E000EA4EC09F0320E096EAB
:10088000060E0A6EC2EC09F0020E096E000EA4EC10
:1008900009F0500E096E060E0A6EC2EC09F0030E46
:1008A000096E000EA4EC09F0C50E116E010E126E59
:1008B0000B0E136E060E146EE1C115F0166AE5C13B
:1008C00017F0186A25EC07F0C50E096E010E0A6EC6
:1008D000C2EC09F0000E0101E46F000EE36F340E6C
:1008E000276EF20EE82EFED7272EFCD70101E34B30
:1008F000E42BE4BFF4D7E45104E1650EE35DD8A036
:10090000EED7899E000EDF6F000EDE6FDFBF06D0D0
:10091000DF512AE1050EDE5DD8B026D08CA202D0D0
:10092000010E01D0000EFF0A276E27468C502718B3
:10093000FD0B27188C6E000EE46F000EE36F340E73
:10094000276EF20EE82EFED7272EFCD70101E34BCF
:10095000E42BE4BFF4D7E45104E1330EE35DD8A007
:10096000EED7DE4BDF2BD2D78C92010E3EEC09F096
:10097000000E83B4010E0101E06FE051D8A462D2F1
:10098000AF05D8A45FD283AE02D0000E1CD083ACDA
:1009900002D0010E18D083AA02D0020E14D083A870
:1009A00002D0030E10D082AE02D0040E0CD082AC66
:1009B00002D0050E08D03004D8B406D082AA02D0E6
:1009C000060E01D00A0EE26F0A0EE219D8B43AD22E
:1009D0007E0EE225D96EDA6A010EDA2228C0DFFF28
:1009E000850EE225D96EDA6A010EDA2229C0DFFF10
:1009F0008C0EE225D96EDA6A010EDA222AC0DFFFF8
:100A0000930EE225D96EDA6A010EDA222BC0DFFFDF
:100A1000690EE225D96EDA6A010EDA222CC0DFFFF8
:100A2000700EE225D96EDA6A010EDA222DC0DFFFE0
:100A3000770EE225D96EDA6A010EDA222EC0DFFFC8
:100A4000200EB26FB2C1B1F1B1C1B0F183511DEC52
:100A500008F00101B36F82511DEC08F00101B46F81
:100A600081511DEC08F00101B56F80511DEC08F0BB
:100A70000101B66F7F511DEC08F00101B76F7E5187
:100A80001DEC08F00101B86F3004D8B405D08451D2
:100A90001DEC08F0010101D0200EB96F200EBB6FD4
:100AA000BBC1BAF18A511DEC08F00101BC6F89513C
:100AB0001DEC08F00101BD6F88511DEC08F001012B
:100AC000BE6F87511DEC08F00101BF6F86511DEC10
:100AD00008F00101C06F85511DEC08F00101C16FE4
:100AE0003004D8B405D08B511DEC08F0010101D0C1
:100AF000200EC26F000EC36F200E9C6F9CC19BF135
:100B00009BC19AF191511DEC08F001019D6F90512C
:100B10001DEC08F001019E6F8F511DEC08F00101E2
:100B20009F6F8E511DEC08F00101A06F8D511DECDF
:100B300008F00101A16F8C511DEC08F00101A26FBA
:100B40003004D8B405D092511DEC08F0010101D059
:100B5000200EA36F200EA56FA5C1A4F198511DEC26
:100B600008F00101A66F97511DEC08F00101A76F75
:100B700096511DEC08F00101A86F95511DEC08F08D
:100B80000101A96F94511DEC08F00101AA6F935166
:100B90001DEC08F00101AB6F3004D8B405D09951B9
:100BA0001DEC08F0010101D0200EAC6F000EAD6FFE
:100BB000040E3018D8B408D0050E3018D8B404D0BC
:100BC000030E3018D8A456D0200EC76FC7C1C6F187
:100BD000C6C1C5F175511DEC08F00101C86F745113
:100BE0001DEC08F00101C96F73511DEC08F0010103
:100BF000CA6F72511DEC08F00101CB6F71511DECF1
:100C000008F00101CC6F70511DEC08F00101CD6FAF
:100C1000200ECE6F030E3018D8A429D0200ED16F2D
:100C2000D1C1D0F1D0C1CFF17C511DEC08F0010150
:100C3000D26F7B511DEC08F00101D36F7A511DEC8E
:100C400008F00101D46F79511DEC08F00101D56F56
:100C500078511DEC08F00101D66F77511DEC08F0BA
:100C60000101D76F200ED86F000ED96F05D0000E8E
:100C7000CF6F02D0000EC56F200E566F56C155F1D2
:100C800055C154F16E511DEC08F00101576F6D51C3
:100C90001DEC08F00101586F6C511DEC08F00101CA
:100CA000596F6B511DEC08F001015A6F6A511DEC30
:100CB00008F001015B6F69511DEC08F001015C6FE8
:100CC000200E5D6FE551D8B42FD081A202D0310E35
:100CD00001D0300EDA6F81A602D0310E01D0300E75
:100CE000DB6F80A802D0310E01D0300EDC6F81A006
:100CF00002D0310E01D0300EDD6F5E0E116E010E8E
:100D0000126E420E136E060E146EDAC115F0166ADC
:100D1000DBC117F0186ADCC119F01A6ADDC11BF0DB
:100D20001C6A25EC07F002D0000E5E6FB00E056E57
:100D3000010E066E000E076E010E086EF7EC08F04D
:100D400005500610D8B415D0000E056E010E066EC3
:100D5000B00E076E010E086E61EC09F0000E096E10
:100D6000000EA4EC09F0B00E096E010E0A6EC2EC82
:100D700009F09A0E056E010E066E150E076E010E35
:100D8000086EF7EC08F005500610D8B415D0150E13
:100D9000056E010E066E9A0E076E010E086E61EC6E
:100DA00009F0010E096E000EA4EC09F09A0E096E0E
:100DB000010E0A6EC2EC09F0C50E056E010E066E3C
:100DC0002A0E076E010E086EF7EC08F005500610AB
:100DD000D8B415D02A0E056E010E066EC50E076E2C
:100DE000010E086E61EC09F0020E096E000EA4EC13
:100DF00009F0C50E096E010E0A6EC2EC09F0540E20
:100E0000056E010E066E3F0E076E010E086EF7ECC2
:100E100008F005500610D8B415D03F0E056E010E2F
:100E2000066E540E076E010E086E61EC09F0030E9B
:100E3000096E000EA4EC09F0540E096E010E0A6E44
:100E4000C2EC09F0E0C1AFF193D5150E226E000E91
:100E5000236EE0D0250E2618D8B409D011C0D9FFD2
:100E600012C0DAFF26C0DFFF114A122AD3D0000ECB
:100E70001E6E4DD022C0D9FF23C0DAFFDECF20F096
:100E8000DDCF21F0020E2226000E23222050211059
:100E9000D8A41ED05A0E206E060E216E19D020C086
:100EA000F6FF21C0F7FFF86A11C0D9FF12C0DAFFC0
:100EB000050EF76403D00800F55005D0F6CFE9FF22
:100EC000F7CFEAFFEF50DF6E204A212A114A122A9B
:100ED00020C0F6FF21C0F7FFF86A050EF76403D0C3
:100EE0000800F55005D0F6CFE9FFF7CFEAFFEF5045
:100EF0000009D8B48FD0D3D722C0D9FF23C0DAFFDE
:100F0000DF50266E020E2226000E2322A7D713C022
:100F1000F6FF14C0F7FF134A142A0800F5CF26F095
:100F20002650000AD8B482D0630AD8B4E5D7070A9D
:100F3000D8B407D00D0AD8B404D01A0AD8B49AD7B6
:100F40008DD722C0D9FF23C0DAFFDECF24F0DDCF5A
:100F500025F0020E2226000E232225AE06D0030E17
:100F60001E12246C251ED8B0252A010E266E26508E
:100F7000020D010EF324F66E060EF420F76E090042
:100F8000F550245C0900F5502558D8A005D0262A34
:100F9000050E2618D8A4EBD71EC01DF0030E1D1693
:100FA000D8B408D011C0D9FF12C0DAFF2D0EDF6E01
:100FB000114A122A26C01FF029D01F50020D010E1F
:100FC000F324F66E060EF420F76E0900F5CF07F055
:100FD0000A00F5CF08F024C005F025C006F0A6EC05
:100FE00008F005C00CF006C00DF0000E0F6E0A0EE2
:100FF0000E6E83EC09F00C50300F266E11C0D9FF35
:1010000012C0DAFF26C0DFFF114A122A1F061F286E
:10101000D8A4D3D713C0F6FF14C0F7FF134A142A7D
:101020000800F5CF26F02650D8A414D711C0D9FF58
:1010300012C0DAFF000EDF6E1200056E21D0300EF6
:101040001DD0310E1BD0320E19D0330E17D0340EF6
:1010500015D0350E13D0360E11D0370E0FD0380EF6
:101060000DD0390E0BD0200E09D03B0E07D03A0E12
:1010700005D02D0E03D0250E01D03F0E066E32D0C6
:101080000550000AD8B4DBD7010AD8B4DAD7030A6E
:10109000D8B4D9D7010AD8B4D8D7070AD8B4D7D783
:1010A000010AD8B4D6D7030AD8B4D5D7010AD8B420
:1010B000D4D70F0AD8B4D3D7010AD8B4D2D7030AE9
:1010C000D8B4D1D7010AD8B4D0D7070AD8B4CFD76B
:1010D000010AD8B4CED7030AD8B4CDD7010AD8B400
:1010E000C2D7CBD7065012008390809C8290960E78
:1010F000CFEC08F0300EDEEC09F000D000D01DEC93
:101100000AF0290ECFEC08F01DEC0AF0010ECFEC2E
:1011100008F01DEC0AF0F6EC09F0200EDEEC09F008
:1011200000D000D01DEC0AF0F6EC09F0010E3EEC08
:1011300009F0280E3EEC09F0080E3EEC09F0060E10
:101140003EEC09F00C0E3EEC09F01200000E0A6EA7
:10115000000E096E07500810D8B41CD0010E0B6E9B
:1011600004D0D890073608360B2A08AEFAD7D890A4
:1011700009360A360750055C08500658D8A005D035
:101180000750055E0850065A0980D8900832073289
:101190000B2EEDD709C005F00AC006F01200086E4C
:1011A000000E0A6E000E096E14D0000E0C6E000EBA
:1011B0000B6E0D0EE82EFED700F00B4A0C2A0CBE6B
:1011C000F8D70C5004E10A0E0B5CD8A0F2D7094AFC
:1011D0000A2A0850056E066A0550095C0A50800A02
:1011E000076E0650800A0758D8B01200DED704D028
:1011F000054A062A074A082A07C0D9FF08C0DAFFAD
:10120000DF50096E05C0D9FF06C0DAFFDF500A6E55
:1012100009500A5C0B6E0B50D8A407D005C0D9FF4B
:1012200006C0DAFFDF50D8A4E3D70B50056E066A7C
:1012300005BE06061200086EF6EC09F00850F00B29
:10124000076E0750DEEC09F0050EE82EFED700F021
:10125000809C838000D000D000D000D01DEC0AF02C
:10126000083A0850F00B076E0750DEEC09F0050E47
:10127000E82EFED700F01DEC0AF01200086EF6EC26
:1012800009F00850F00B076E0750DEEC09F0050E70
:10129000E82EFED700F0809C839000D000D000D0D4
:1012A00000D01DEC0AF0083A0850F00B076E07500A
:1012B000DEEC09F0050EE82EFED700F01DEC0AF07A
:1012C000120005C009F006C00AF004D0094A0A2A33
:1012D000074A082A07C0F6FF08C0F7FFF86A09C0E6
:1012E000D9FF0AC0DAFF050EF76403D00800F550F5
:1012F00005D0F6CFE9FFF7CFEAFFEF50DF6EDF5002
:10130000D8B41200E3D70E500F10D8B418D0010E85
:10131000106E04D0D8900E360F36102A0FAEFAD7C2
:101320000E500C5C0F500D58D8A004D00E500C5E1F
:101330000F500D5AD8900F320E32102EF1D70CC02C
:101340000CF00DC00DF012000A6E130E0A6408D0E6
:1013500012000A8C12D0140E01D0540E0A260DD0A1
:101360000950000AD8B409D0010AD8B4F2D7030A48
:10137000D8B4F1D7010AD8B4F0D70A8E0A503EEC9F
:1013800009F0120009C0F6FF0AC0F7FFF86A050E5F
:10139000F76403D00800F55005D0F6CFE9FFF7CF8A
:1013A000EAFFEF500B6E06D00B501BEC09F0094A18
:1013B0000A2AE8D70B50D8B41200F6D7056E05C03C
:1013C00006F006A802D0828201D0829206AA02D03C
:1013D000828401D0829406AC02D0828601D08296AB
:1013E00006AE02D0828801D0829812009488839041
:1013F000808C1DEC0AF00D0EE82EFED700F0000EDA
:101400008BB8010E056E1DEC0AF00550D8A4EED77E
:10141000809C9498140EE82EFED712000101E56B13
:1014200000EE28F0090EEE6AE806FDE131903192F7
:10143000000EF86E000133EF03F08280040EE82EF8
:06144000FED782901200AD
:020000040020DA
:08000000FFFFFFFFFFFFFFFF00
:020000040030CA
:0E000000FF281F3CFFBF85FF0FC00FE00F4021
:00000001FF
